:100000000428FF3FFF3FFF3F9420000083167E300F
:100010009B00B521A40083122408123C031D1D2857
:1000200005191D28E42105191D28E42105191D289D
:10003000E42105191D28E421352FE8210618F22DA9
:10004000E4210618F22DE4210618F22D00008C2779
:1000500086152016A0122013A0135F20E421201281
:100060005F20E42120165F20E42120125F20E4219C
:1000700020165F20E42120165F20E82120125F2057
:10008000E82120165F20E82120125F20E8212016B9
:100090005F20E82120125F20E82120165F20201237
:1000A000A0122017A0135F20A010CD210B22201634
:1000B000A0122013A0135F20181218166F2A631EB7
:1000C0006728201E652806126C2806166C28201E3C
:1000D0006B2806166C280612E31E7428A01E7228D0
:1000E0008612792886167928A01E782886167928FF
:1000F0008612631F8128201F7F2806138628061773
:100100008628201F8528061786280613E31F8E28B9
:10011000A01F8C288613932886179328A01F922847
:100120008617932886130800831303138312003065
:100130008B0000308C0000309000003092000030C6
:10014000970007309F00B030980083168030810000
:1001500000308C0000308E0000309F00243098006A
:1001600040309900243085000730860083128501D5
:100170008601831600309B00B521E000B521E20026
:10018000B521E300B521E400B521E500B521E60085
:10019000B521AA00A0015F20F030A0005F20E4217B
:1001A000A0015F20E0080319E00A6008E100EF0108
:1001B000E701E8016A21ED01403084008001840AF2
:1001C0000408503C031DDE284030840024308000A9
:1001D000840A50308000840A53308000840A5230F0
:1001E0008000840A46308000840A31308000840A0E
:1001F00030308000840A36308000840A2C30800041
:10020000840A2A08013C031D172931308000840A22
:1002100037308000840A38308000840A2A30800019
:10022000840A33308000840A3230800067292A082B
:10023000023C031D2D2931308000840A37308000B4
:10024000840A39308000840A2A308000840A3330DE
:100250008000840A3330800067292A08033C031D8C
:10026000432931308000840A38308000840A3030DD
:100270008000840A2A308000840A33308000840A97
:100280003530800067292A08043C031D5929313084
:100290008000840A38308000840A31308000840A6B
:1002A0002A308000840A33308000840A3430800091
:1002B000672932308000840A31308000840A2A3075
:1002C0008000840A30308000840A463080000000BC
:1002D000AC010800EA01EB01EC016408023C031DDB
:1002E00083296808EB000310EB0CEC0C0310EB0CFB
:1002F000EC0C0310EB0CEC0C6718EA14E7186A1509
:100300006719EA15B4296408043C031D9729680895
:10031000EB000310EB0CEC0C0310EB0CEC0C67186F
:100320006B17E718EA1467196A15EA11B42964080B
:10033000083C031DA8296808EB000310EB0CEC0C2B
:100340006718EB17E718EA1467196A15EA11B42958
:100350006408103C031D71296808EB006718EA1453
:10036000E7186A15EA11B429080083161C149B0AC1
:100370001A088312080083167F309B00AA309A0067
:10038000C12983161C1555309D00AA309D009C1470
:100390009C18C8291C1183120800403084000008F2
:1003A000A100003C0319D729DE21840ACF290D3092
:1003B000A100DE210A30A100DE21080083120C1EFC
:1003C000DF29210899000800E821E821E821E82137
:1003D0006330A500F321A50BEA29F62100000800EF
:1003E000000000000000000000000000F830A40041
:1003F0000000000000000000000000000000A40B4E
:10040000F8290000000000000000000000000000CB
:100410000000000008001725201C0B2A2308243C9C
:10042000031D6D2A1725201C122A2308413C031D99
:100430006D2A1725201C192A2308633C031D6D2AE9
:100440001725201C202A23086B3C031D6D2A172525
:10045000201C272A2308203C031D6D2A1725201C59
:100460002E2A2308493C031D6D2A1725201C352AF6
:1004700023086E3C031D6D2A1725201C3C2A2308E7
:10048000703C031D6D2A1725201C432A2308753C48
:10049000031D6D2A1725201C4A2A2308743C031DBE
:1004A0006D2A1725201C512A2308313C031D6D2A73
:1004B0001725201C582A2308303C031D6D2A1725B8
:1004C000201C5F2A2308363C031D6D2A1725201C9B
:1004D000662A23082E3C03196E2A0B2A0800000006
:1004E0002C1C05102C10503084008001840A040854
:1004F000603C031D752A1725201C7B2A2308243CF9
:10050000031D7B2A1725201C822A2308473C031D34
:100510007B2A1725201C892A2308503C031D7B2A8F
:100520001725201C902A2308473C031D7B2A1725EA
:10053000201C972A2308473C031D7B2A1725201CD3
:100540009E2A2308413C031D7B2A1725201CA52A2F
:1005500023082C3C031D122D05101725201CAD2A45
:1005600023185016A318D0161725201CB42A2318B8
:100570005014A318D01423195015A319D0151725FA
:10058000201CBF2A23185116A318D116231951175E
:100590001725201CC82A23185114A318D114231975
:1005A0005115A319D1151725201CD32A231852162B
:1005B000A318D21623195217A319D2171725201CD6
:1005C000DE2A23185214A318D21423195215A31982
:1005D000D2151725201CE92A23082E3C031D122DB5
:1005E0001725201CF02A23185316A318D3162319F5
:1005F0005317A319D3171725201CFB2A23185314AC
:10060000A318D31423195315A319D3151725201C88
:10061000062B23185416A318D41623195417A319FC
:10062000D4171725201C112B23082C3C031D122D39
:100630001725201C182B23185414A318D41423197D
:100640005415A319D4151725201C232B2318551630
:10065000A318D51623195517A319D5171725201C2C
:100660002E2B23185514A318D51423195515A31987
:10067000D5151725201C392B23185616A318D61666
:1006800023195617A319D6171725201C442B230806
:100690002E3C031D122D1725201C4B2B23185614FE
:1006A000A318D61423195615A319D6151725201CDF
:1006B000562B23185716A318D71623195717A31903
:1006C000D7171725201C612B23185714A318D714EC
:1006D00023195715A319D7151725201C6C2B231880
:1006E0005816A318D81623195817A319D817172561
:1006F000201C772B23082C3C031D122D1725201CB2
:100700007E2B23084E3C031D872BD0178C2B2308F0
:10071000533C031D122DD0131725201C8C2B2308AE
:100720002C3C031D122D1725201C932B2318D815A4
:100730001725201C982B23185916A318D9162319EE
:100740005917A319D9171725201CA32B231859149F
:10075000A318D91423195915A319D9151725201C25
:10076000AE2B23185A16A318DA1623195A17A319F1
:10077000DA171725201CB92B23185A14A318DA14DA
:1007800023195A15A319DA151725201CC42B230881
:100790002E3C031D122D1725201CCB2B23185B1676
:1007A000A318DB1623195B17A319DB171725201CC9
:1007B000D62B23185B14A318DB1423195B15A3197C
:1007C000DB151725201CE12B23185C16A318DC165B
:1007D00023195C17A319DC171725201CEC2B2318F1
:1007E0005C14A318DC1423195C15A319DC15172558
:1007F000201CF72B23082C3C031D122D1725201C31
:10080000FE2B2308453C031D072C50170C2C2308F6
:10081000573C031D122D50131725201C0C2C2308A8
:100820002C3C031D122D1725201C132C2318D11727
:100830001725201C182C23082C3C031D122D1725CE
:10084000201C1F2C2308313C031958151725201C88
:10085000262C23185D16A318DD1623195D17A3197E
:10086000DD171725201C312C23082C3C031D122DCD
:100870001725201C382C1725201C3B2C1725201C45
:100880003E2C23082E3C031D122D1725201C452C21
:100890001725201C482C23082C3C031D122D17253E
:1008A000201C4F2C1725201C522C23185D14A31834
:1008B000DD1423195D15A319DD151725201C5D2CEA
:1008C00023185E16A318DE1623195E17A319DE1768
:1008D0001725201C682C23185E14A318DE14231976
:1008E0005E15A319DE151725201C732C23185F161F
:1008F000A318DF1623195F17A319DF171725201C6C
:100900007E2C23082E3C031D122D1725201C852C20
:1009100023185F14A318DF1423195F15A319DF151B
:100920001725201C902C23082C3C031D122D172565
:10093000201C972C23084D3C031D122D0618A92CB2
:100940000618A92C0618A92C0618A92C2C08803AE0
:10095000AC00D11FAD2CAC1B0514A01620135F20DA
:10096000AB0AAB18B52C8510B62C85141725201CA6
:10097000B62C2308243C031DB62C1725201CBD2CA7
:100980002308473C031D122D1725201CC42C2308C7
:10099000503C031D122D1725201CCB2C2308473C4F
:1009A000031D122D1725201CD22C2308533C031D98
:1009B000122D1725201CD92C2308413C031D122D74
:1009C000AC1B05141725201CE22C23082C3C031D0E
:1009D000122D1725201CE92C2308413C031D122D44
:1009E0001725201CF02C23082C3C031D122D172545
:1009F000201CF72C230823185814A318D814D11F2F
:100A0000032DD818052DA0100D2DA01C0B2DE10BCA
:100A10000D2D6008E1002625A014A0125F201812F9
:100A200018166F2AA01220135F20A0106F2A201022
:100A3000031383128C1E252D1A08A3002014981C62
:100A4000252DA0175F20181218160800ED08031DA9
:100A50002A2D6625503084000008E9000927201956
:100A60002E2D840A0408603C031D2C2DED0A6D0810
:100A70006402031D652D20175F202C14D125ED0184
:100A80000030EF006808013EE8000318E70A6A2119
:100A900067086502031D652D68086602031D652D44
:100AA000E208031D602D8611BB210510A012201342
:100AB000A01320165F20E72120125F20E721592D87
:100AC000E701E8016A21E408ED000800A725A0304D
:100AD000E900EA18E9146A196915EA19E9157D258A
:100AE00020196F2D6B08E9007D252019742D6C08E5
:100AF000E9007D252019792D0800E91F812DC325E6
:100B0000822DB525691F862DC325872DB525E91EA4
:100B10008B2DC3258C2DB525691E902DC325912DB8
:100B2000B525E91D952DC325962DB525691D9A2D51
:100B3000C3259B2DB525E91C9F2DC325A02DB525CB
:100B4000691CA42DC325A52DB525DF250800051694
:100B500000000000000085150000000000000512E4
:100B600000000000000085110800051200000000D0
:100B70000000851500000000000085110000000045
:100B80000000051208000516000000000000851591
:100B900000000000000085110000000000000512A8
:100BA000080005120000000000008515000000008C
:100BB00000000516000000000000851108008316E3
:100BC000343085008312332785153427051AEA2D22
:100BD0002011EB2D20158511332783162430850035
:100BE00083120800EF08031D7F2E2012A012201789
:100BF000A0135F20E701E801ED01F626F6266A2141
:100C00002430A100DE216408023C031D122EE901FC
:100C1000E6266B08E900EA19E9176A196917EA1864
:100C2000E916382E6408043C031D1F2EE9016A19D9
:100C30006914E6266B08E900EA18E917382E6408FB
:100C4000083C031D2C2EE9016A19E914EA186914FD
:100C5000E6266B08E900382E6408103C031D072EB9
:100C6000E9016A19E914EA186914E6266B08E90033
:100C7000E6266C08E900E626F62666250F30A70072
:100C8000201B442E2017452E20135F209526A226D8
:100C90000512332785153427851133270516E626D7
:100CA000A70B472EA2260516332785153427851155
:100CB0003327D125E626F626ED0A6D086402031DCA
:100CC0003E2EED016808013EE8000318E70A6A219C
:100CD00067086502031DFF2D68086602031DFF2DCE
:100CE0002430A100DE214530A100DE214E30A100DC
:100CF000DE214430A100DE21F626EF0A942E6F0893
:100D0000023C0319942EEF0A2430A100DE21443066
:100D1000A100DE214F30A100DE214E30A100DE21F6
:100D20004530A100DE21F6260528A725A130E900DF
:100D3000EA18E9146A196915EA19E9150927201949
:100D40009E2E0800E90105168316343085008312B3
:100D5000332785153427051AE91700008511332735
:100D600085153427051A6917000085113327851565
:100D70003427051AE9160000851133278515342715
:100D8000051A691600008511332785153427051AC1
:100D9000E91500008511332785153427051A6915D3
:100DA00000008511332785153427051AE914000042
:100DB0008511332785153427051A6914000085111C
:100DC000332783162430850083120800690E0F39FB
:100DD000A900FD262908A800A100DE2169080F3915
:100DE000A900FD262908A100DE2108000D30A10080
:100DF000DE210A30A100DE2108002908093C031C7D
:100E0000052F2908303EA900082F2908373EA900E0
:100E10000800E91F0D2FC3250E2FB525691F122FBE
:100E2000C325132FB525E91E172FC325182FB52568
:100E3000691E1C2FC3251D2FB525E91D212FC32594
:100E4000222FB525691D262FC325272FB525E91C7F
:100E50002B2FC3252C2FB525691C302FC325312FEF
:100E6000B525DF25080008000800ED01E701E801CD
:100E7000A601A0122013A01320125F20503084007E
:100E8000FF308000840A0408603C031D402FED08F9
:100E9000031D4B2F6625503084000008E900092708
:100EA00020194F2F840A0408603C031D4D2FA60A09
:100EB000261E5E2FA01220132012612FA0162017CD
:100EC00020165F20ED0A6D086402031D8B2FD125CB
:100ED000ED01F021F021F021F021F021F021F021AD
:100EE000F021F021F021F0216808013EE80003180C
:100EF000E70A6A2167086502031D8B2F68086602EE
:100F0000031D8B2F20122013A0165F20E721A012B3
:100F10005F20E721842F472F0000E701E8016A21C5
:100F200066259526A22605163327851534278511B3
:100F30003327D1256908FF3C0319BB2F6808013E00
:100F4000E8000318E70A6A2167086502031D8F2F6E
:100F500068086602031D8F2FE208031DB92FA01237
:100F60002013A013E82120165F20E82120125F2023
:100F7000B22FE701E8010800FF3FFF3FFF3FFF3FBF
:100F8000FF3FFF3FFF3FFF3FFF3FFF3FFF3FFF3F71
:100F9000FF3FFF3FFF3FFF3FFF3FFF3FFF3FFF3F61
:100FA000FF3FFF3FFF3FFF3FFF3FFF3FFF3FFF3F51
:100FB000FF3FFF3FFF3FFF3FFF3FFF3FFF3FFF3F41
:1042000001000000F0001000040000000000FF00AA
:10421000FF00FF00FF00FF00FF00FF00FF00FF00A6
:10422000FF00FF00FF00FF00FF00FF00FF00FF0096
:10423000FF00FF00FF00FF00FF00FF00FF00FF0086
:10424000FF00FF00FF00FF00FF00FF00FF00FF0076
:10425000FF00FF00FF00FF00FF00FF00FF00FF0066
:10426000FF00FF00FF00FF00FF00FF00FF00FF0056
:10427000FF00FF00FF00FF00FF00FF00FF00FF0046
:10428000FF00FF00FF00FF00FF00FF00FF00FF0036
:10429000FF00FF00FF00FF00FF00FF00FF00FF0026
:1042A000FF00FF00FF00FF00FF00FF00FF00FF0016
:1042B000FF00FF00FF00FF00FF00FF00FF00FF0006
:1042C000FF00FF00FF00FF00FF00FF00FF00FF00F6
:1042D000FF00FF00FF00FF00FF00FF00FF00FF00E6
:1042E000FF00FF00FF00FF00FF00FF00FF00FF00D6
:1042F000FF00FF00FF00FF00FF00FF001200FF00B3
:10430000FF00FF00FF00FF00FF00FF00FF00FF00B5
:10431000FF00FF00FF00FF00FF00FF00FF00FF00A5
:10432000FF00FF00FF00FF00FF00FF00FF00FF0095
:10433000FF00FF00FF00FF00FF00FF00FF00FF0085
:10434000FF00FF00FF00FF00FF00FF00FF00FF0075
:10435000FF00FF00FF00FF00FF00FF00FF00FF0065
:10436000FF00FF00FF00FF00FF00FF00FF00FF0055
:10437000FF00FF00FF00FF00FF00FF00FF00FF0045
:10438000FF00FF00FF00FF00FF00FF00FF00FF0035
:10439000FF00FF00FF00FF00FF00FF00FF00FF0025
:1043A000FF00FF00FF00FF00FF00FF00FF00FF0015
:1043B000FF00FF00FF00FF00FF00FF00FF00FF0005
:1043C000FF00FF00FF00FF00FF00FF00FF00FF00F5
:1043D000FF00FF00FF00FF00FF00FF00FF00FF00E5
:1043E000FF00FF00FF00FF00FF00FF00FF00FF00D5
:1043F000FF00FF00FF00FF00FF00FF00FF00FF00C5
:1080000001000000F0001000040000000000FF006C
:10801000FF00FF00FF00FF00FF00FF00FF00FF0068
:10802000FF00FF00FF00FF00FF00FF00FF00FF0058
:10803000FF00FF00FF00FF00FF00FF00FF00FF0048
:10804000FF00FF00FF00FF00FF00FF00FF00FF0038
:10805000FF00FF00FF00FF00FF00FF00FF00FF0028
:10806000FF00FF00FF00FF00FF00FF00FF00FF0018
:10807000FF00FF00FF00FF00FF00FF00FF00FF0008
:10808000FF00FF00FF00FF00FF00FF00FF00FF00F8
:10809000FF00FF00FF00FF00FF00FF00FF00FF00E8
:1080A000FF00FF00FF00FF00FF00FF00FF00FF00D8
:1080B000FF00FF00FF00FF00FF00FF00FF00FF00C8
:1080C000FF00FF00FF00FF00FF00FF00FF00FF00B8
:1080D000FF00FF00FF00FF00FF00FF00FF00FF00A8
:1080E000FF00FF00FF00FF00FF00FF00FF00FF0098
:1080F000FF00FF00FF00FF00FF00FF001200FF0075
:10810000FF00FF00FF00FF00FF00FF00FF00FF0077
:10811000FF00FF00FF00FF00FF00FF00FF00FF0067
:10812000FF00FF00FF00FF00FF00FF00FF00FF0057
:10813000FF00FF00FF00FF00FF00FF00FF00FF0047
:10814000FF00FF00FF00FF00FF00FF00FF00FF0037
:10815000FF00FF00FF00FF00FF00FF00FF00FF0027
:10816000FF00FF00FF00FF00FF00FF00FF00FF0017
:10817000FF00FF00FF00FF00FF00FF00FF00FF0007
:10818000FF00FF00FF00FF00FF00FF00FF00FF00F7
:10819000FF00FF00FF00FF00FF00FF00FF00FF00E7
:1081A000FF00FF00FF00FF00FF00FF00FF00FF00D7
:1081B000FF00FF00FF00FF00FF00FF00FF00FF00C7
:1081C000FF00FF00FF00FF00FF00FF00FF00FF00B7
:1081D000FF00FF00FF00FF00FF00FF00FF00FF00A7
:1081E000FF00FF00FF00FF00FF00FF00FF00FF0097
:1081F000FF00FF00FF00FF00FF00FF00FF00FF0087
:08400000F03FF83FF03FF53FEF
:02400E00223F4F
:10401000FF3FFF3FFF3FFF3FFF3FFF3FFF3FFF3FB0
:00000001FF
